:100000000C94460018950000189500001895000003
:10001000189500001895000018950000189500002C
:10002000189500001895000018950000189500001C
:10003000189500001895000018950000189500000C
:1000400018950000189500000C94072518950000DD
:1000500018950000189500001895000018950000EC
:1000600018950000189500001895000018950000DC
:1000700018950000189500001895000018950000CC
:100080001895000018950000189500008FEF8DBF9F
:10009000C8EDE0EC4E2E80E48EBFD0E4F0E45F2E9D
:1000A000A89584B7082E877F84BF88E1992780931D
:1000B000600090936000EEEFFFE3A0E0B1E08827DE
:1000C0008D933197E9F70E94482766248CE00E94BF
:1000D0009627E2EFF0E00E94A52B80E40E9496278D
:1000E00058E0D895802D0E94902731965A95C9F7EF
:1000F00004C01F1F1F1F20202020EAE1F1E00E9402
:10010000A52B88E40E94962758E0D895802D0E9460
:10011000902731965A95C9F704C0202020201F1F30
:100120001F1FE2E4F1E00E94A52B80E50E949627C4
:1001300058E0D895802D0E94902731965A95C9F79E
:1001400004C01F1F1F1F1F1F1F1FEAE6F1E00E94B0
:10015000A52B88E50E94962758E0D895802D0E940F
:10016000902731965A95C9F704C006090906202040
:100170002020E2E9F1E00E94A52B80E60E9496276C
:1001800058E0D895802D0E94902731965A95C9F74E
:1001900004C002040E010F110F20EAEBF1E00E94EF
:1001A000A52B88E60E94962758E0D895802D0E94BE
:1001B000902731965A95C9F704C00A200E111111E3
:1001C0000E20E2EEF1E00E94A52B80E70E94962728
:1001D00058E0D895802D0E94902731965A95C9F7FE
:1001E00004C008040E111F100E20EAE0F2E00E9485
:1001F000A52B88E70E94962758E0D895802D0E946D
:10020000902731965A95C9F704C00A20111111118F
:100210000E2085E085BD80E084BD3F983E983D98E6
:100220003C983A98209A219A239A509A519A529A35
:10023000539A549A569A3B9A089A099A559A81EC7D
:100240008093800081E08093810088E290E0A3E0C9
:10025000B1E08D939C938CE390E0A1E0B1E08D93AD
:100260009C938AE0809305010091050148E0049F7A
:10027000A6E0B1E00C92A1E0B1E00D911C914AE939
:1002800050E0040F151F802F912F909389008093C9
:100290008800479A469A459A449A70917C017F7DDE
:1002A00070937C0180E08093E70170917C017F7BFB
:1002B00070937C0180E08093F40181E08093DB0106
:1002C00080E080934A018CE080934B0181E0809331
:1002D0004C018CE080934D0182E080934E0180E0E0
:1002E00080934F0180E08093500180E08093510122
:1002F00081E08093DD0181E08093E80170917C01D1
:10030000777F70937C0181E0809382010E942D278A
:100310008FE711E00E943C27E2E8FAE50E94A52B56
:100320000E9426278FEB11E00E943C27EEE8FAE5B9
:100330000E94A52B0E94262785E00E949027E2E9D3
:10034000FAE50E94A52B0E94262786E00E949027AE
:10035000E6E9FAE50E94A52B0E94262781E080931A
:100360007D0100917D01083518F011F00C941F02F9
:10037000ADE7B1E0EC91FF27ADE7B1E0AD90BB2474
:10038000A2E8B1E0AA0DBB1D91E00E94562CADE79A
:10039000B1E0AD90BB24A2E8B1E0AA0DBB1D0C9169
:1003A0000F3F11F00C94DE0180E0ADE7B1E0AD90BD
:1003B000BB24A2E8B1E0AA0DBB1D8C9300917D0186
:1003C00048E00E945D2CA5EEB1E08C930091E50120
:1003D000003011F00C94F60180E0ADE7B1E0AD9093
:1003E000BB24A2E8B1E0AA0DBB1D8C9300917D0156
:1003F00044E00E945D2CA0EEB1E00C930091E0017E
:10040000003018F011F00C9407020C94130283EDE5
:10041000A0EEB1E01C910E943C27EAE9FAE50E94B7
:10042000A52B0E94262784E190E00E94DC27ADE7FF
:10043000B1E08C918F5F8C9310F40C94B101E4E6E1
:10044000F0E0A3E0B1E092E00E94562CA3E0B1E01E
:100450000D911C910F3F50E0150711F00C943602DE
:1004600088E290E0A3E0B1E08D939C93E5E6F0E0B4
:10047000A4EFB1E091E00E94562C0091F4010F3FEF
:1004800011F00C94460280E08093F401E6E6F0E07F
:10049000A1EFB1E091E00E94562C0091F1010F3FD5
:1004A00011F00C94560280E08093F101E7E6F0E051
:1004B000A7EFB1E091E00E94562C0091F7010F3FA9
:1004C00011F00C94660280E08093F7010E942D27C2
:1004D00087E0E9E20E94692BA5E1B2E00C93ECE928
:1004E000FAE50E94A52B0E94262786E00E9490270D
:1004F000E0EAFAE50E94A52B0E94262785E00E94EB
:100500009027E4EAFAE50E94A52B0E94262784E0C2
:100510000E949027EAEAFAE50E94A52B0E9426276E
:10052000A8EAB0E4E5E1F2E00E94CB2B0E94192793
:1005300084EF91E00E94DC270E942D270091150294
:10054000003018F011F00C94A7020C94B10387E06E
:10055000E9E20E94F42AA4E0B2E0EAE1F2E098E0E5
:100560000E94372C87E0E9E20E94F92AACE0B2E071
:10057000EAE1F2E098E00E94372C00910B02003093
:1005800011F00C94D80270917C01706270937C0120
:100590008FE711E00E943C27E0EBFAE50E94A52BD3
:1005A0000E94262784EF91E00E94DC270C943103FF
:1005B00087E0E4E0F2E00E946D2C402F00910B02F6
:1005C000041711F00C941E038FE711E00E943C27E2
:1005D000E2ECFAE50E94A52B0E94262784EF91E029
:1005E0000E94DC278FE711E00E943C27E6EDFAE548
:1005F0000E94A52B0E94262781E08093140200917F
:100600001402083018F011F00C941C03A8EAB0E4AE
:10061000E4E1F2E0A190BB24E3E0F2E0EA0DFB1D8F
:100620000E94152C0E941927A4E1B2E08C918F5FE3
:100630008C9310F40C94FF020C94310370917C01A4
:10064000706270937C018FE711E00E943C27ECED13
:10065000FAE50E94A52B0E94262784EF91E00E94D4
:10066000DC2784EF91E00E94DC2740911302009187
:100670000B02041711F00C94520370917C0170610D
:1006800070937C018FEB11E00E943C27E0EFFAE5CC
:100690000E94A52B0E94262784EF91E00E94DC2770
:1006A0000C94AB0387E0ECE0F2E00E946D2C402F4D
:1006B00000911302041711F00C9498038FEB11E0D2
:1006C0000E943C27E2E0FBE50E94A52B0E94262722
:1006D00084EF91E00E94DC278FEB11E00E943C2721
:1006E000E6E1FBE50E94A52B0E94262781E080938E
:1006F000140200911402083018F011F00C949603C3
:10070000A8EAB0E4E4E1F2E0A190BB24EBE0F2E07F
:10071000EA0DFB1D0E94152C0E941927A4E1B2E0EE
:100720008C918F5F8C9310F40C9479030C94AB0331
:1007300070917C01706170937C018FEB11E00E94DD
:100740003C27ECEDFAE50E94A52B0E94262784EFBA
:1007500091E00E94DC2784EF91E00E94DC270C945A
:10076000B60370917C01706270937C01ACE7B1E0DC
:100770008C9185FB16F00C94D20383ED11E00E945E
:100780003C27ECE1FBE50E94A52B0E94262735992A
:100790000C94CC030C94D20382E390E00E94DC27FB
:1007A0000C94BD030E942D278FE711E00E943C2787
:1007B000E0E3FBE50E94A52B0E94262786E00E942D
:1007C0009027E2E3FBE50E94A52B0E94262708E084
:1007D0000E9421278FEB11E00E943C27A8EAB0E499
:1007E000ECE3FBE50E94A52B0E94F5270E94192748
:1007F00083E911E00E943C27E0E5FBE50E94A52B80
:100800000E94262783ED11E00E943C27E6E6FBE5E7
:100810000E94A52B0E94262786E00E949027EAE6E8
:10082000FBE50E94A52B0E9426270E945623E1E0AB
:10083000F0E00E943F270E946523A9EFB1E08D916F
:100840009C91AEE7B1E08D939C93A9EFB1E08D91BF
:100850009C91A0E8B1E08D939C93E1E0F0E00E94D0
:100860003F2780E08093140280E080931502789403
:1008700070916E00716070936E000E942D270E942F
:10088000562380E080931502009115020A3018F07B
:1008900011F00C946F040E94E6190E94951D3D987A
:1008A000ACE7B1E09C9192FF04C0359B10C09B7FE8
:1008B0009C9335990CC08AE09F9399270E94DC276E
:1008C0009F91359904C094609C930E947504A5E1A2
:1008D000B2E08C918F5F8C9310F40C9444040E94CE
:1008E00065230C943F04F894FFCF0E942D2781E0EC
:1008F00080937B0100917B01043018F011F00C947F
:1009000083040C94860481E080937B013C98ACE7DF
:10091000B1E09C9191FF04C0349B10C09D7F9C93DB
:1009200034990CC08AE09F9399270E94DC279F91FD
:10093000349904C092609C930E9407063E98ACE7ED
:10094000B1E09C9190FF04C0369B10C09E7F9C93A9
:1009500036990CC08AE09F9399270E94DC279F91CB
:10096000369904C091609C930E940D063F98A2E2C4
:10097000B2E09C9197FF04C0379B10C09F779C9377
:1009800037990CC08AE09F9399270E94DC279F919A
:10099000379904C090689C930C94040600917B01E5
:1009A000013011F00C941D058FE711E00E943C27E7
:1009B000EAE7FBE50E94A52B0E94262784E00E941F
:1009C0009027E8E8FBE50E94A52B0E94262786E9F0
:1009D00090E00E94DC273F98A2E2B2E09C9197FF52
:1009E00004C0379B10C09F779C9337990CC08AE056
:1009F0009F9399270E94DC279F91379904C09068A4
:100A00009C930C9404063D98ACE7B1E09C9192FF56
:100A100004C0359B10C09B7F9C9335990CC08AE025
:100A20009F9399270E94DC279F91359904C0946079
:100A30009C930E9405080C940206023011F00C945D
:100A400061058FE711E00E943C27E0E9FBE50E9489
:100A5000A52B0E94262786E990E00E94DC273F987C
:100A6000A2E2B2E09C9197FF04C0379B10C09F7731
:100A70009C9337990CC08AE09F9399270E94DC27AA
:100A80009F91379904C090689C930C9404063D98FC
:100A9000ACE7B1E09C9192FF04C0359B10C09B7FF6
:100AA0009C9335990CC08AE09F9399270E94DC277C
:100AB0009F91359904C094609C930E943F180C94B8
:100AC0000206033011F00C94AE058FE711E00E948E
:100AD0003C27E4EAFBE50E94A52B0E94262784E040
:100AE0000E949027E4EBFBE50E94A52B0E9426279D
:100AF00086E990E00E94DC273F98A2E2B2E09C9158
:100B000097FF04C0379B10C09F779C9337990CC008
:100B10008AE09F9399270E94DC279F91379904C010
:100B200090689C930C9404063D98ACE7B1E09C91CE
:100B300092FF04C0359B10C09B7F9C9335990CC0DD
:100B40008AE09F9399270E94DC279F91359904C0E2
:100B500094609C930E940E0D0C940206043011F0D8
:100B60000C9402068FE711E00E943C27EAEBFBE5BC
:100B70000E94A52B0E94262784E00E949027E4EC87
:100B8000FBE50E94A52B0E94262784E00E94902767
:100B9000EAECFBE50E94A52B0E94262786E990E05F
:100BA0000E94DC273F98A2E2B2E09C9197FF04C02C
:100BB000379B10C09F779C9337990CC08AE09F9316
:100BC00099270E94DC279F91379904C090689C93D5
:100BD0000C9404063D98ACE7B1E09C9192FF04C0F0
:100BE000359B10C09B7F9C9335990CC08AE09F93E6
:100BF00099270E94DC279F91359904C094609C93AB
:100C00000E9413060C947A040E942D270895ABE7E6
:100C1000B1E08C918F5F8C93089580917B0181501E
:100C200080937B0108950E942D2781E080937B01B2
:100C300000917B01053018F011F00C9421060C9402
:100C4000240681E080937B013C98ACE7B1E09C9165
:100C500091FF04C0349B10C09D7F9C9334990CC0BD
:100C60008AE09F9399270E94DC279F91349904C0C2
:100C700092609C930E9407063E98ACE7B1E09C917D
:100C800090FF04C0369B10C09E7F9C9336990CC089
:100C90008AE09F9399270E94DC279F91369904C090
:100CA00091609C930E940D063F98A2E2B2E09C9155
:100CB00097FF04C0379B10C09F779C9337990CC057
:100CC0008AE09F9399270E94DC279F91379904C05F
:100CD00090689C930C94040800917B01013011F002
:100CE0000C94B2068FE711E00E943C27E0EDFBE593
:100CF0000E94A52B0E94262786E990E00E94DC270F
:100D00003F98A2E2B2E09C9197FF04C0379B10C0CD
:100D10009F779C9337990CC08AE09F9399270E94F4
:100D2000DC279F91379904C090689C930C94040829
:100D30003D98ACE7B1E09C9192FF04C0359B10C098
:100D40009B7F9C9335990CC08AE09F9399270E94C2
:100D5000DC279F91359904C094609C930E940814ED
:100D60000C940208023011F00C9408078FE711E090
:100D70000E943C27E4EEFBE50E94A52B0E9426275B
:100D800084E00E949027E2EFFBE50E94A52B0E94E1
:100D9000262785E00E949027E8EFFBE50E94A52B1F
:100DA0000E94262786E990E00E94DC273F98A2E275
:100DB000B2E09C9197FF04C0379B10C09F779C9333
:100DC00037990CC08AE09F9399270E94DC279F9156
:100DD000379904C090689C930C9404083D98ACE744
:100DE000B1E09C9192FF04C0359B10C09B7F9C9307
:100DF00035990CC08AE09F9399270E94DC279F9128
:100E0000359904C094609C930E94BB140C94020812
:100E1000033011F00C946A078FE711E00E943C2721
:100E2000EAEFFBE50E94A52B0E94262785E00E94A1
:100E3000902786E00E949027E4E0FCE50E94A52B25
:100E40000E94262786E00E949027E0EAFAE50E94A9
:100E5000A52B0E94262785E00E949027E8EFFBE55E
:100E60000E94A52B0E94262786E990E00E94DC279D
:100E70003F98A2E2B2E09C9197FF04C0379B10C05C
:100E80009F779C9337990CC08AE09F9399270E9483
:100E9000DC279F91379904C090689C930C940408B8
:100EA0003D98ACE7B1E09C9192FF04C0359B10C027
:100EB0009B7F9C9335990CC08AE09F9399270E9451
:100EC000DC279F91359904C094609C930E94D515AE
:100ED0000C940208043011F00C94AE078FE711E077
:100EE0000E943C27E8E0FCE50E94A52B0E942627F3
:100EF00086E990E00E94DC273F98A2E2B2E09C9154
:100F000097FF04C0379B10C09F779C9337990CC004
:100F10008AE09F9399270E94DC279F91379904C00C
:100F200090689C930C9404083D98ACE7B1E09C91C8
:100F300092FF04C0359B10C09B7F9C9335990CC0D9
:100F40008AE09F9399270E94DC279F91359904C0DE
:100F500094609C930E94B4160C940208053011F022
:100F60000C9402088FE711E00E943C27ECE1FCE5BD
:100F70000E94A52B0E94262785E00E949027E4E28C
:100F8000FCE50E94A52B0E94262785E00E94902761
:100F9000E8E2FCE50E94A52B0E94262786E990E066
:100FA0000E94DC273F98A2E2B2E09C9197FF04C028
:100FB000379B10C09F779C9337990CC08AE09F9312
:100FC00099270E94DC279F91379904C090689C93D1
:100FD0000C9404083D98ACE7B1E09C9192FF04C0EA
:100FE000359B10C09B7F9C9335990CC08AE09F93E2
:100FF00099270E94DC279F91359904C094609C93A7
:101000000E946A170C941806089581E080937B0172
:1010100070917C017F7770937C013D98ACE7B1E0E3
:101020009C9192FF04C0359B10C09B7F9C93359987
:101030000CC08AE09F9399270E94DC279F913599E5
:1010400004C094609C930E9407063F98A2E2B2E01D
:101050009C9197FF04C0379B10C09F779C93379952
:101060000CC08AE09F9399270E94DC279F913799B3
:1010700004C090689C930C940D0D00917B0101308D
:1010800011F00C949D088FE711E00E943C27E2E3E9
:10109000FCE50E94A52B0E9426270E942B0C83E9C9
:1010A00011E00E943C27AFE2B1E00E941B27E4E47C
:1010B000FCE50E94A52B0E942627A8E3B1E00E9430
:1010C0001B2783ED11E00E943C27E8E4FCE50E9429
:1010D000A52B0E94262702E10E94212734990C9417
:1010E0008608AFE1B1E08C918F5F8C9300911F0176
:1010F000073118F011F00C947F080C94820880E0FE
:1011000080931F0186E990E00E94DC2736990C94B9
:101110009B0880911F01815080931F0100911F0146
:101120000F3F11F00C94970887E180931F0186E927
:1011300090E00E94DC270C94290C023011F00C94F2
:10114000FE088FE711E00E943C27ECE4FCE50E94DA
:10115000A52B0E9426270E942B0C83E911E00E94F8
:101160003C27AFE2B1E00E941B27E4E4FCE50E94CB
:10117000A52B0E942627A8E3B1E00E941B2783ED40
:1011800011E00E943C2703E00E942127E8E4FCE5EF
:101190000E94A52B0E9426270FE00E942127349948
:1011A0000C94E708AEE1B1E08C918F5F8C930091D5
:1011B0001E010B3318F011F00C94E0080C94E308B6
:1011C00080E080931E0186E990E00E94DC2736993A
:1011D0000C94FC0880911E01815080931E010091A7
:1011E0001E010F3F11F00C94F8088BE380931E0151
:1011F00086E990E00E94DC270C94290C033011F062
:101200000C945F098FE711E00E943C27E0E6FCE5C3
:101210000E94A52B0E9426270E942B0C83E911E037
:101220000E943C27AFE2B1E00E941B27E4E4FCE50A
:101230000E94A52B0E942627A8E3B1E00E941B274D
:1012400083ED11E00E943C2706E00E942127E8E49C
:10125000FCE50E94A52B0E9426270CE00E94212776
:1012600034990C944809A4E1B1E08C918F5F8C9380
:10127000009114010B3318F011F00C9441090C94F7
:10128000440980E08093140186E990E00E94DC2705
:1012900036990C945D09809114018150809314015A
:1012A000009114010F3F11F00C9459098BE38093C6
:1012B000140186E990E00E94DC270C94290C04308C
:1012C00011F00C94BD098FE711E00E943C27E0E784
:1012D000FCE50E94A52B0E9426270E942B0C83E987
:1012E00011E00E943C27AFE2B1E00E941B27E4E43A
:1012F000FCE50E94A52B0E942627A8E3B1E00E94EE
:101300001B2783ED11E00E943C270AE00E94212761
:10131000E4E8FCE50E94A52B0E94262734990C9452
:10132000A609A5E2B1E08C918F5F8C930091250115
:101330000E3018F011F00C949F090C94A2098CE067
:101340008093250186E990E00E94DC2736990C9471
:10135000BB098091250181508093250100912501D1
:101360000B3011F00C94B7098EE08093250186E9CB
:1013700090E00E94DC270C94290C053011F00C94AD
:101380001B0A8FE711E00E943C27EAE8FCE50E9477
:10139000A52B0E9426270E942B0C83E911E00E94B6
:1013A0003C27AFE2B1E00E941B27E4E4FCE50E9489
:1013B000A52B0E942627A8E3B1E00E941B2783EDFE
:1013C00011E00E943C270FE00E942127E8E4FCE5A1
:1013D0000E94A52B0E94262734990C94040AA4E2AB
:1013E000B1E08C918F5F8C93009124010C3018F048
:1013F00011F00C94FD090C94000A81E08093240103
:1014000086E990E00E94DC2736990C94190A8091B5
:10141000240181508093240100912401003011F0B7
:101420000C94150A8CE08093240186E990E00E94D8
:10143000DC270C94290C063011F00C94790A8FE704
:1014400011E00E943C27EEE9FCE50E94A52B0E94DA
:1014500026270E942B0C83E911E00E943C27AFE273
:10146000B1E00E941B27E4E4FCE50E94A52B0E944A
:101470002627A8E3B1E00E941B2783ED11E00E941C
:101480003C2702E10E942127E8E4FCE50E94A52B0D
:101490000E94262734990C94620AA2E2B1E08C9152
:1014A0008F5F8C93009122010F3118F011F00C9492
:1014B0005B0A0C945E0A81E08093220186E990E049
:1014C0000E94DC2736990C94770A80912201815082
:1014D0008093220100912201003011F00C94730AD4
:1014E0008FE18093220186E990E00E94DC270C9432
:1014F000290C073011F00C947E0B8FE711E00E944D
:101500003C27E2EBFCE50E94A52B0E94262783E9FD
:1015100011E00E943C2700912301003011F00C944F
:10152000A90AE4ECFCE50E94A52B0E9426270FE007
:101530000E94212783ED11E00E943C27EAECFCE5A4
:101540000E94A52B0E9426270FE00E9421270C94C1
:101550004F0B013011F00C94C50AE0EDFCE50E9440
:10156000A52B0E94262700E10E94212783ED11E090
:101570000E943C27E4E8FCE50E94A52B0E94262758
:1015800000E10E9421270C944F0B023011F00C94C3
:10159000E10AE6EDFCE50E94A52B0E9426270EE05D
:1015A0000E94212783ED11E00E943C27EEEDFCE52F
:1015B0000E94A52B0E9426270EE00E9421270C9452
:1015C0004F0B033011F00C94FD0AE6EEFCE50E948F
:1015D000A52B0E9426270BE00E94212783ED11E016
:1015E0000E943C27E0EFFCE50E94A52B0E942627E5
:1015F0000BE00E9421270C944F0B043011F00C9447
:10160000190BEAEFFCE50E94A52B0E9426270EE0AD
:101610000E94212783ED11E00E943C27EEEDFCE5BE
:101620000E94A52B0E9426270EE00E9421270C94E1
:101630004F0B053011F00C94350BE2E0FDE50E94F4
:10164000A52B0E9426270DE00E94212783ED11E0A3
:101650000E943C27EAE0FDE50E94A52B0E94262778
:101660000DE00E9421270C944F0B063011F00C94D2
:101670004F0BE2E1FDE50E94A52B0E9426270CE01E
:101680000E94212783ED11E00E943C27ECE1FDE55B
:101690000E94A52B0E9426270CE00E942127349946
:1016A0000C94670BA3E2B1E08C918F5F8C93009157
:1016B0002301063018F011F00C94600B0C94630BAE
:1016C00080E08093230186E990E00E94DC27369930
:1016D0000C947C0B80912301815080932301009115
:1016E00023010F3F11F00C94780B86E080932301C7
:1016F00086E990E00E94DC270C94290C083011F058
:101700000C94EC0B8FE711E00E943C27E6E2FDE52C
:101710000E94A52B0E9426270BE00E94212783E927
:1017200011E00E943C2703E00E942127EEE2FDE544
:101730000E94A52B0E94262709E00E94212783ED05
:1017400011E00E943C27ACE7B1E08C9187FB16F0DA
:101750000C94B80B03E00E942127E4E8FCE50E940A
:10176000A52B0E9426270FE00E9421270C94C40B72
:1017700009E00E942127E8E3FDE50E94A52B0E94D5
:10178000262708E00E942127A6E2B0E00C9104FB86
:1017900081E00EF480E08F93A6E2B0E00C9106FBAE
:1017A00081E00EF480E09F91892B882311F40C9442
:1017B000EA0BACE7B1E08C9187FB882780F9809534
:1017C00080FBACE7B1E08C9187F98C9386E990E0DF
:1017D0000E94DC270C94290C093011F00C94290C80
:1017E000ACE7B1E08C9187FB16F00C940D0C0E94D5
:1017F000011B0E942D278FEB11E00E943C27ECE398
:10180000FDE50E94A52B0E942627E2E0F0E00E9461
:101810003F270E943D040C94290C0E942D278FEB3A
:1018200011E00E943C27EAE4FDE50E94A52B0E94FE
:10183000262783E911E00E943C27EAECFCE50E94A0
:10184000A52B0E942627E2E0F0E00E943F270E949D
:101850003D040C940D08A1E4B1E0EFE1F1E00E9439
:10186000CB2BE1E4F1E0A8EAB0E40E94312CE8EAF5
:10187000F0E4A1E4B1E01127222702E033270E941F
:10188000022AE1E4F1E0AFE2B1E00E94312CAFE2E4
:10189000B1E00E941227EAE5FDE50E94A52B0E9417
:1018A000F527A1E4B1E0EEE1F1E00E94CB2BE1E409
:1018B000F1E0A8EAB0E40E94312CE8EAF0E4A1E407
:1018C000B1E01127222702E033270E94022AE1E437
:1018D000F1E0AFE2B1E00E9412270E94312CAFE2AA
:1018E000B1E00E941227EAE5FDE50E94A52B0E94C7
:1018F000F527A1E4B1E0E4E1F1E00E94CB2BE1E4C3
:10190000F1E0A8EAB0E40E94312CE8EAF0E4A1E4B6
:10191000B1E01127222702E033270E94022AE1E4E6
:10192000F1E0AFE2B1E00E9412270E94312CA1E465
:10193000B1E0E5E2F1E00E94CB2BE1E4F1E0A8EABE
:10194000B0E40E94312CE8EAF0E4A1E4B1E0112710
:10195000222702E033270E94022AA8E3B1E0ECE547
:10196000FDE50E94A52B0E94F527E1E4F1E0A8E344
:10197000B1E00E9412270E94312CA8E3B1E00E943E
:101980001227E0E6FDE50E94A52B0E94F527A1E4C1
:10199000B1E0E4E2F1E00E94CB2BE1E4F1E0A8EA5F
:1019A000B0E40E94312CE8EAF0E4A1E4B1E01127B0
:1019B000222702E033270E94022AE1E4F1E0A8E3B3
:1019C000B1E00E9412270E94312CA8E3B1E00E94EE
:1019D0001227E0E6FDE50E94A52B0E94F527A1E471
:1019E000B1E0E2E2F1E00E94CB2BE1E4F1E0A8EA11
:1019F000B0E40E94312CE8EAF0E4A1E4B1E0112760
:101A0000222702E033270E94022AE1E4F1E0A8E362
:101A1000B1E00E9412270E94312C089581E080934A
:101A20007B0170917C017F7770937C013D98ACE7DE
:101A3000B1E09C9192FF04C0359B10C09B7F9C93AA
:101A400035990CC08AE09F9399270E94DC279F91CB
:101A5000359904C094609C930E9407063F98A2E2C7
:101A6000B2E09C9197FF04C0379B10C09F779C9376
:101A700037990CC08AE09F9399270E94DC279F9199
:101A8000379904C090689C930C94021400917B01D8
:101A9000013011F00C94630E8FE711E00E943C2797
:101AA000E2E6FDE50E94A52B0E94262705E00E94A4
:101AB00021270E949C130E9413138FEB11E00E94B8
:101AC0003C27E2E7FDE50E94A52B0E942627A8EA15
:101AD000B0E4EBEDF1E00E94CB2B0E94192703E06C
:101AE0000E9421278FEB1BE00E943C2700914A01B6
:101AF000003011F00C94840DEAE7FDE50E94A52B5F
:101B00000E9426270C948A0DE2E8FDE50E94A52B91
:101B10000E94262783E91BE00E943C270091500188
:101B2000003011F00C949C0DECE8FDE50E94A52B13
:101B30000E9426270C94080EE6E9FDE50E94A52BDD
:101B40000E94262700914F01003011F00C94B90D2E
:101B5000ECE9FDE50E94A52B0E94262786E00E9465
:101B60009027EEE9FDE50E94A52B0E9426270C9404
:101B7000080E013011F00C94C50DE2EAFDE50E945B
:101B8000A52B0E9426270C94080E023011F00C940D
:101B9000D10DE8EAFDE50E94A52B0E9426270C94B2
:101BA000080E033011F00C94DD0DEEEAFDE50E9405
:101BB000A52B0E9426270C94080E043011F00C94DB
:101BC000F20DE4EBFDE50E94A52B0E94262786E09E
:101BD0000E949027E6EBFDE50E94A52B0E94262798
:101BE0000C94080E053011F00C94FE0DEAEBFDE5A7
:101BF0000E94A52B0E9426270C94080E063011F097
:101C00000C94080EE0ECFDE50E94A52B0E9426270F
:101C100083ED11E00E943C27E6ECFDE50E94A52B38
:101C20000E942627A0E6B1E00E941B2704E00E9444
:101C3000212783ED1DE00E943C27EAECFDE50E9490
:101C4000A52B0E942627A9E6B1E00E941B2783E965
:101C500017E00E943C27EAE9FAE50E94A52B0E94C2
:101C6000262734990C944B0EABEDB1E08C918F5F2D
:101C70008C93409105010091DB01041718F011F0DD
:101C80000C94440E0C94470E81E08093DB0186E9AE
:101C900090E00E94DC2736990C94610E8091DB0164
:101CA00081508093DB010091DB01003011F00C9436
:101CB0005D0E809105018093DB0186E990E00E9432
:101CC000DC270C941113023011F00C94E00E8FEB12
:101CD00011E00E943C2704E10E9421278FE711E0D8
:101CE0000E943C27A8EAB0E4EBEDF1E00E94CB2B88
:101CF0000E941927EEECFDE50E94A52B0E942627E5
:101D000008E00E94212783E911E00E943C2703E0BC
:101D10000E942127EEE2FDE50E94A52B0E942627C6
:101D200009E00E94212783ED11E00E943C270091E9
:101D30004A01013011F00C94AB0E03E00E94212700
:101D4000E4E8FCE50E94A52B0E9426270DE00E94F6
:101D500021270C94B70E09E00E942127E8E3FDE556
:101D60000E94A52B0E94262708E00E942127A6E2B8
:101D7000B0E00C9104FB81E00EF480E08F93A6E2CA
:101D8000B0E00C9106FB81E00EF480E09F91892B7E
:101D9000882311F40C94DE0E00914A01003011F0FA
:101DA0000C94D70E81E080934A010C94DA0E80E007
:101DB00080934A0186E990E00E94DC270C9411137D
:101DC000033011F00C945C0F00914A01003011F0C7
:101DD0000C94ED0E89E080937B018FE711E00E9467
:101DE0003C27A8EAB0E4EBEDF1E00E94CB2B0E9487
:101DF0001927ECEDFDE50E94A52B0E94262783E91B
:101E000011E00E943C2703E00E942127E0EFFDE55E
:101E10000E94A52B0E94262707E00E94212783ED20
:101E200011E00E943C2700915001003011F00C9409
:101E3000270F03E00E942127E4E8FCE50E94A52B80
:101E40000E9426270DE00E9421270C94330F09E001
:101E50000E942127E4E8FCE50E94A52B0E9426278A
:101E600007E00E942127A6E2B0E00C9104FB81E08C
:101E70000EF480E08F93A6E2B0E00C9106FB81E0C7
:101E80000EF480E09F91892B882311F40C945A0F53
:101E900000915001003011F00C94530F81E08093B9
:101EA00050010C94560F80E08093500186E990E039
:101EB0000E94DC270C941113043011F00C94D60FFF
:101EC0008FE711E00E943C27A8EAB0E4EBEDF1E0D7
:101ED0000E94CB2B0E941927ECEFFDE50E94A52B59
:101EE0000E94262704E00E9421278FEB11E00E9428
:101EF0003C2700915001003011F00C94870FECE06A
:101F0000FEE50E94A52B0E9426270C948D0FE2E18E
:101F1000FEE50E94A52B0E9426270E94131383E949
:101F200011E00E943C27A0E6B1E00E941B270FE0D1
:101F30000E94212783ED11E00E943C27E8E4FCE5A4
:101F40000E94A52B0E94262702E10E942127349996
:101F50000C94BF0FABE4B1E08C918F5F8C93009138
:101F60004B01073118F011F00C94B80F0C94BB0F13
:101F700080E080934B0186E990E00E94DC2736994F
:101F80000C94D40F80914B01815080934B010091B0
:101F90004B010F3F11F00C94D00F87E180934B0160
:101FA00086E990E00E94DC270C941113053011F0B3
:101FB0000C9450108FE711E00E943C27A8EAB0E48F
:101FC000EBEDF1E00E94CB2B0E941927ECEFFDE531
:101FD0000E94A52B0E94262704E00E9421278FEB58
:101FE00011E00E943C2700915001003011F00C9448
:101FF0000110ECE0FEE50E94A52B0E9426270C9420
:102000000710E2E1FEE50E94A52B0E9426270E9410
:10201000131383E911E00E943C27A0E6B1E00E947F
:102020001B2783ED11E00E943C2703E00E9421273B
:10203000E8E4FCE50E94A52B0E9426270FE00E9401
:10204000212734990C943910ACE4B1E08C918F5F66
:102050008C9300914C010B3318F011F00C9432105A
:102060000C94351080E080934C0186E990E00E944A
:10207000DC2736990C944E1080914C01815080934E
:102080004C0100914C010F3F11F00C944A108BE36E
:1020900080934C0186E990E00E94DC270C94111398
:1020A000063011F00C94CA108FE711E00E943C2713
:1020B000A8EAB0E4EBEDF1E00E94CB2B0E941927D7
:1020C000E8E1FEE50E94A52B0E94262704E00E947D
:1020D00021278FEB11E00E943C2700915001003036
:1020E00011F00C947B10ECE0FEE50E94A52B0E9401
:1020F00026270C948110E2E1FEE50E94A52B0E94A8
:1021000026270E94131383E911E00E943C27A9E6C9
:10211000B1E00E941B270FE00E94212783ED11E010
:102120000E943C27E8E4FCE50E94A52B0E9426279C
:1021300002E10E94212734990C94B310ADE4B1E080
:102140008C918F5F8C9300914D01073118F011F045
:102150000C94AC100C94AF1080E080934D0186E994
:1021600090E00E94DC2736990C94C81080914D01B4
:10217000815080934D0100914D010F3F11F00C945F
:10218000C41087E180934D0186E990E00E94DC272E
:102190000C941113073011F00C9444118FE711E0E7
:1021A0000E943C27A8EAB0E4EBEDF1E00E94CB2BC3
:1021B0000E941927E8E1FEE50E94A52B0E94262730
:1021C00004E00E9421278FEB11E00E943C27009140
:1021D0005001003011F00C94F510ECE0FEE50E9487
:1021E000A52B0E9426270C94FB10E2E1FEE50E943D
:1021F000A52B0E9426270E94131383E911E00E9459
:102200003C27A9E6B1E00E941B2783ED11E00E9464
:102210003C2703E00E942127E8E4FCE50E94A52B6F
:102220000E9426270FE00E94212734990C942D113B
:10223000AEE4B1E08C918F5F8C9300914E010B3333
:1022400018F011F00C9426110C94291180E0809361
:102250004E0186E990E00E94DC2736990C944211E9
:1022600080914E01815080934E0100914E010F3FAD
:1022700011F00C943E118BE380934E0186E990E0BF
:102280000E94DC270C941113083011F00C945D129D
:1022900000915001003011F00C94511189E08093AD
:1022A0007B018FE711E00E943C27A8EAB0E4EBED48
:1022B000F1E00E94CB2B0E941927E8E2FEE50E9484
:1022C000A52B0E94262704E00E94212783E911E024
:1022D0000E943C2700914F01003011F00C948811AE
:1022E000E4ECFCE50E94A52B0E9426270FE00E944B
:1022F000212783ED11E00E943C27EAECFCE50E94D7
:10230000A52B0E9426270FE00E9421270C942E1255
:10231000013011F00C94A411E0EDFCE50E94A52B16
:102320000E94262700E10E94212783ED11E00E94F0
:102330003C27E4E8FCE50E94A52B0E94262700E14B
:102340000E9421270C942E12023011F00C94C0111F
:10235000E6EDFCE50E94A52B0E9426270EE00E94D8
:10236000212783ED11E00E943C27EEEDFCE50E9461
:10237000A52B0E9426270EE00E9421270C942E12E6
:10238000033011F00C94DC11E6EEFCE50E94A52B65
:102390000E9426270BE00E94212783ED11E00E9476
:1023A0003C27E0EFFCE50E94A52B0E9426270BE0CE
:1023B0000E9421270C942E12043011F00C94F81175
:1023C000EAEFFCE50E94A52B0E9426270EE00E9462
:1023D000212783ED11E00E943C27EEEDFCE50E94F1
:1023E000A52B0E9426270EE00E9421270C942E1276
:1023F000053011F00C941412E2E0FDE50E94A52BCB
:102400000E9426270DE00E94212783ED11E00E9403
:102410003C27EAE0FDE50E94A52B0E9426270DE05F
:102420000E9421270C942E12063011F00C942E12CB
:10243000E2E1FDE50E94A52B0E9426270CE00E9408
:10244000212783ED11E00E943C27ECE1FDE50E948D
:10245000A52B0E9426270CE00E94212734990C947A
:102460004612AFE4B1E08C918F5F8C9300914F01E5
:10247000063018F011F00C943F120C94421280E0D8
:1024800080934F0186E990E00E94DC2736990C94F6
:102490005B1280914F01815080934F0100914F0159
:1024A0000F3F11F00C94571286E080934F0186E99C
:1024B00090E00E94DC270C941113093011F00C9469
:1024C000D2128FE711E00E943C27E8E3FEE50E946C
:1024D000A52B0E9426270CE00E9421278FEB11E0FC
:1024E0000E943C2705E00E94212783E911E00E9419
:1024F0003C2703E00E942127EEE2FDE50E94A52B88
:102500000E94262708E00E94212783ED11E00E9407
:102510003C27ACE7B1E08C9187FB16F00C949E123F
:1025200003E00E942127E4E8FCE50E94A52B0E941D
:1025300026270CE00E9421270C94AA1209E00E9491
:102540002127E8E3FDE50E94A52B0E94262707E04E
:102550000E942127A6E2B0E00C9104FB81E00EF47A
:1025600080E08F93A6E2B0E00C9106FB81E00EF4D0
:1025700080E09F91892B882311F40C94D012ACE752
:10258000B1E08C9187FB882780F9809580FBACE7D0
:10259000B1E08C9187F98C9386E990E00E94DC276A
:1025A0000C9411130A3011F00C941113ACE7B1E044
:1025B0008C9187FB16F00C94F4120E947C1B0E94F5
:1025C0002D278FEB11E00E943C27ECE3FDE50E94F4
:1025D000A52B0E942627E2E0F0E00E943F2781E041
:1025E00080937B010C9411130E942D278FEB11E037
:1025F0000E943C27EAE4FDE50E94A52B0E942627C5
:1026000083E911E00E943C27EAECFCE50E94A52B3F
:102610000E942627E2E0F0E00E943F2781E08093BD
:102620007B010C94160DA2E7B1E0EBE4F1E00E940F
:10263000CB2BE2E7F1E0A8EAB0E40E94312CE8EA13
:10264000F0E4A2E7B1E01127222702E033270E943D
:10265000022AE2E7F1E0A0E6B1E00E94312CA0E618
:10266000B1E00E941227EAE5FDE50E94A52B0E9439
:10267000F527A2E7B1E0ECE4F1E00E94CB2BE2E722
:10268000F1E0A8EAB0E40E94312CE8EAF0E4A2E725
:10269000B1E01127222702E033270E94022AE2E755
:1026A000F1E0A0E6B1E00E9412270E94312CA2E7DF
:1026B000B1E0EDE4F1E00E94CB2BE2E7F1E0A8EA23
:1026C000B0E40E94312CE8EAF0E4A2E7B1E011277F
:1026D000222702E033270E94022AE2E7F1E0A9E67E
:1026E000B1E00E94312CA9E6B1E00E941227EAE590
:1026F000FDE50E94A52B0E94F527A2E7B1E0EEE4DC
:10270000F1E00E94CB2BE2E7F1E0A8EAB0E40E94FE
:10271000312CE8EAF0E4A2E7B1E01127222702E039
:1027200033270E94022AE2E7F1E0A9E6B1E00E9425
:1027300012270E94312C08950091DB0141E0041B17
:10274000ACEDB1E00C93ACEDB1E00C9148E0049F2E
:102750000C92ACEDB1E0AD90BB24A3E8B1E0AA0DC2
:10276000BB1D8C9180934A01ACEDB1E0AD90BB24D0
:10277000A4E8B1E0AA0DBB1D8C9180934B01ACED98
:10278000B1E0AD90BB24A5E8B1E0AA0DBB1D8C91D2
:1027900080934C01ACEDB1E0AD90BB24A6E8B1E074
:1027A000AA0DBB1D8C9180934D01ACEDB1E0AD90B5
:1027B000BB24A7E8B1E0AA0DBB1D8C9180934E010C
:1027C000ACEDB1E0AD90BB24A8E8B1E0AA0DBB1D13
:1027D0008C9180934F01ACEDB1E0AD90BB24A9E8A2
:1027E000B1E0AA0DBB1D8C9180935001ACEDB1E01E
:1027F000AD90BB24AAE8B1E0AA0DBB1D8C918093DB
:10280000510108950E942D2781E080937B01089556
:10281000A1E0B1E08D919C91A2EFB1E08D939C93EA
:102820008FE711E00E943C27E2E4FEE50E94A52B21
:102830000E94262783E911E00E943C27E8E5FEE597
:102840000E94A52B0E942627A8EAB0E4E1E0F1E06F
:102850000E94C42B0E941927E4E6FEE50E94A52BE6
:102860000E942627A8EAB0E4E2EFF1E00E94C42B20
:102870000E94192734990C945414A1E0B1E00E94ED
:10288000C426A1E0B1E00D911C91043650E015077B
:102890001CF011F00C944E140C94541480E090E051
:1028A000A1E0B1E08D939C9336990C946C14A1E057
:1028B000B1E00E94CB26A1E0B1E00D911C91003067
:1028C00050E015070CF402C00C946C1484E690E000
:1028D000A1E0B1E08D939C93A1E0B1E00D911C913A
:1028E0004AE950E0040F151F802F912F9093890023
:1028F0008093880086E990E00E94DC273D98ACE751
:10290000B1E09C9192FF04C0359B10C09B7F9C93CB
:1029100035990CC08AE09F9399270E94DC279F91EC
:10292000359904C094609C930C94B8143F98A2E22B
:10293000B2E09C9197FF04C0379B10C09F779C9397
:1029400037990CC08AE09F9399270E94DC279F91BA
:10295000379904C090689C930C94B0140C94101494
:10296000A2EFB1E08D919C91A1E0B1E08D939C9399
:102970000E942D270895A3E0B1E08D919C91A9EECE
:10298000B1E08D939C938FE711E00E943C27E4EE29
:10299000FBE50E94A52B0E94262784E00E94902739
:1029A000E8E6FEE50E94A52B0E94262783E910E0B9
:1029B0000E943C27E0E7FEE50E94A52B0E94262707
:1029C00083E91AE00E943C27E4E7FEE50E94A52B7C
:1029D0000E94262783E911E10E943C27E8E7FEE5F3
:1029E0000E94A52B0E9426278FEB11E00E943C2716
:1029F000EEE7FEE50E94A52B0E94262784E00E94B8
:102A00009027E6E8FEE50E94A52B0E942627A8EA6B
:102A1000B0E4E3E0F1E00E94C42B0E941927E4E651
:102A2000FEE50E94A52B0E94262734990C9443159D
:102A3000A3E0B1E00D911C914AE050E0040F151F96
:102A4000A3E0B1E00D931C93A3E0B1E00D911C91C4
:102A5000043650E015071CF011F00C9431150C945D
:102A6000371580E090E0A3E0B1E08D939C9383ED77
:102A7000A8EEB1E01C910E943C27E8EFFBE50E9424
:102A8000A52B0E94262736990C946F15A3E0B1E080
:102A90000D911C914AE050E0041B150BA3E0B1E03E
:102AA0000D931C93A3E0B1E00D911C91003050E018
:102AB00015070CF402C00C94631584E690E0A3E0C3
:102AC000B1E08D939C9383EDA8EEB1E01C910E9440
:102AD0003C27E8EFFBE50E94A52B0E9426270091EA
:102AE000030145E00E945D2CA8EEB1E00C9300913B
:102AF000E801003011F00C94801581E08093E8012A
:102B000083EDA8EEB1E01C910E943C27ECE8FEE5C5
:102B10000E94A52B0E9426273D98ACE7B1E09C912E
:102B200092FF04C0359B10C09B7F9C9335990CC0CD
:102B30008AE09F9399270E94DC279F91359904C0D2
:102B400094609C930C94CA153F98A2E2B2E09C91C9
:102B500097FF04C0379B10C09F779C9337990CC098
:102B60008AE09F9399270E94DC279F91379904C0A0
:102B700090689C930C94C21586E990E00E94DC2733
:102B80000C94F414A9EEB1E08D919C91A3E0B1E016
:102B90008D939C930E942D27E4E6F0E0A3E0B1E042
:102BA00092E07BE70E94452C08958091F10180938B
:102BB000F0018FE711E00E943C27EAEFFBE50E945D
:102BC000A52B0E94262785E00E94902786E00E9480
:102BD0009027E4E0FCE50E94A52B0E94262786E0D2
:102BE0000E949027E0EAFAE50E94A52B0E94262782
:102BF00085E00E949027E8EFFBE50E94A52B0E944C
:102C000026278FEB11E00E943C27EEE8FEE50E94AC
:102C1000A52B0E94262786E00E949027E4E9FEE586
:102C20000E94A52B0E94262783E911E00E943C27E1
:102C300003E00E942127EEE2FDE50E94A52B0E9401
:102C4000262708E00E94212783ED11E00E943C27FF
:102C50000091F101013011F00C943C1603E00E9448
:102C60002127E4E8FCE50E94A52B0E9426270CE022
:102C70000E9421270C94481609E00E942127E8E3CE
:102C8000FDE50E94A52B0E94262707E00E94212730
:102C9000A6E2B0E00C9104FB81E00EF480E08F939B
:102CA000A6E2B0E00C9106FB81E00EF480E09F917B
:102CB000892B882311F40C946F160091F1010030D8
:102CC00011F00C94681681E08093F1010C946B165E
:102CD00080E08093F10186E990E00E94DC2782E3A6
:102CE00090E00E94DC273D98ACE7B1E09C9192FF18
:102CF00004C0359B10C09B7F9C9335990CC08AE023
:102D00009F9399270E94DC279F91359904C0946076
:102D10009C930C94A9163F98A2E2B2E09C9197FF75
:102D200004C0379B10C09F779C9337990CC08AE0F2
:102D30009F9399270E94DC279F91379904C0906840
:102D40009C930C94A5160C9424168091F00180930A
:102D5000F1010E942D27E6E6F0E0A1EFB1E091E05D
:102D60007BE70E94452C08958091F4018093F50142
:102D70008FE711E00E943C27E8E0FCE50E94A52BCC
:102D80000E94262783E911E00E943C2703E00E946D
:102D90002127ECE9FEE50E94A52B0E94262708E0EA
:102DA0000E94212783ED11E00E943C270091F4014D
:102DB000003011F00C94EA1603E00E942127EEED9A
:102DC000FCE50E94A52B0E9426270AE00E942127ED
:102DD0000C94F6160BE00E942127E4E8FCE50E9423
:102DE000A52B0E94262705E00E942127A6E2B0E03D
:102DF0000C9104FB81E00EF480E08F93A6E2B0E03A
:102E00000C9106FB81E00EF480E09F91892B8823D2
:102E100011F40C941417A4EFB1E08C9180958C936D
:102E200086E990E00E94DC273D98ACE7B1E09C91F8
:102E300092FF04C0359B10C09B7F9C9335990CC0BA
:102E40008AE09F9399270E94DC279F91359904C0BF
:102E500094609C930C944A173F98A2E2B2E09C9134
:102E600097FF04C0379B10C09F779C9337990CC085
:102E70008AE09F9399270E94DC279F91379904C08D
:102E800090689C930C9446170C94D2168091F5018F
:102E90008093F4010091F401013011F00C94551766
:102EA0008BE0809305010C9458178AE0809305010C
:102EB0000091050148E0049FA6E0B1E00C920E9459
:102EC0002D27E5E6F0E0A4EFB1E091E07BE70E947A
:102ED000452C08958091F7018093F8018FE711E068
:102EE0000E943C27ECE1FCE50E94A52B0E942627CE
:102EF00085E00E949027E4E2FCE50E94A52B0E9459
:102F0000262785E00E949027EAEAFEE50E94A52B8D
:102F10000E94262783E911E00E943C2701E00E94DD
:102F20002127E0EBFEE50E94A52B0E94262783EDDA
:102F300011E00E943C270091F701003011F00C9441
:102F4000AF1701E00E942127EAECFCE50E94A52BC7
:102F50000E9426270EE00E9421270C94D1170130F1
:102F600011F00C94C11708E00E942127EAECFCE55F
:102F70000E94A52B0E94262707E00E9421270C947F
:102F8000D117023011F00C94D1170FE00E942127C5
:102F9000E4E8FCE50E94A52B0E94262701E00E94A0
:102FA000212734990C94E917A7EFB1E08C918F5F3A
:102FB0008C930091F701023018F011F00C94E21795
:102FC0000C94E51780E08093F70186E990E00E9479
:102FD000DC2736990C94FE178091F701815080937D
:102FE000F7010091F701003010F00C94FA1782E01D
:102FF0008093F70186E990E00E94DC273D98ACE7DA
:10300000B1E09C9192FF04C0359B10C09B7F9C93C4
:1030100035990CC08AE09F9399270E94DC279F91E5
:10302000359904C094609C930C9434183F98A2E2A4
:10303000B2E09C9197FF04C0379B10C09F779C9390
:1030400037990CC08AE09F9399270E94DC279F91B3
:10305000379904C090689C930C9430180C9497177F
:103060008091F8018093F7010E942D27E7E6F0E0B8
:10307000A7EFB1E091E07BE70E94452C089581E045
:1030800080937B0170917C017F7770937C0180E05D
:103090008093DF0180E080937D0100917D010C3001
:1030A00018F011F00C948018EAE7FDE40E94A52BBB
:1030B000ADE7B1E08C919927A0EEB1E00E94DD2947
:1030C0008FEBA0EEB1E01C910E943C27ECE5FDE403
:1030D0000E94A52BADE7B1E08C9199270E94E829C9
:1030E000A1EEB1E00E94F527A1EEB1E00E941B27FE
:1030F000ADE7B1E08C918F5F8C9310F40C944D1878
:103100003D98ACE7B1E09C9192FF04C0359B10C0A4
:103110009B7F9C9335990CC08AE09F9399270E94CE
:10312000DC279F91359904C094609C930E945819A4
:103130003F98A2E2B2E09C9197FF04C0379B10C079
:103140009F779C9337990CC08AE09F9399270E94A0
:10315000DC279F91379904C090689C930E94C11905
:1031600000917B01013011F00C9456198FE711E0AA
:103170000E943C27E2E6FDE50E94A52B0E9426273F
:1031800005E00E94212783E911E00E943C2704E129
:103190000E942127EAE7FDE40E94A52BAFEDB1E0F4
:1031A0008C919927A0EEB1E00E94DD2983E9A0EE81
:1031B000B1E01C910E943C2783E00E94902700917F
:1031C000E0010A3011F00C94F318A0EEB1E08C91FC
:1031D0008F5F8C9383E9A0EEB1E01C910E943C27A5
:1031E00083E00E9490270091E0010F3011F00C94D1
:1031F0000719A0EEB1E08C918F5F8C9383E9A0EE6C
:10320000B1E01C910E943C2783E00E94902700912E
:10321000E001023111F00C942919A0EEB1E08C917B
:103220008F5F8C9383E9A0EEB1E01C910E943C2754
:1032300083E00E949027A0EEB1E08C918F5F8C9389
:1032400083E9A0EEB1E01C910E943C2783E00E943C
:10325000902734990C944119AFEDB1E08C918F5FB8
:103260008C930091DF010C3018F011F00C943A1996
:103270000C943D1980E08093DF0186E990E00E9484
:10328000DC2736990C9456198091DF018150809388
:10329000DF010091DF010F3F11F00C9452198CE017
:1032A0008093DF0186E990E00E94DC270C9480186F
:1032B0000091DF01003011F00C94621981E083B9B4
:1032C0000C94C019013011F00C946A1982E083B992
:1032D0000C94C019023011F00C94721988E083B973
:1032E0000C94C019033011F00C947A1981E089B95B
:1032F0000C94C019043011F00C94821982E089B941
:103300000C94C019053011F00C948A1984E089B925
:103310000C94C019063011F00C94921988E089B908
:103320000C94C019073011F00C949A1980E189B9F6
:103330000C94C019083011F00C94A21980E489B9DA
:103340000C94C019093011F00C94AA1988E086B9C0
:103350000C94C0190A3011F00C94B2190E94D019C3
:103360000C94C0190B3011F00C94BA1981E080B99B
:103370000C94C0190C3011F00C94C01982E080B983
:103380000895289829982B98589859985A985B9896
:103390005C985E984398109811980E943D04089597
:1033A00081E083B982E083B988E083B981E089B99B
:1033B00082E089B984E089B988E089B980E189B976
:1033C00080E489B988E086B9089508950E94E92CBF
:1033D00010EA0E94012D12E00E94012D0E94E92CAA
:1033E00011EA0E94012D0E94202DA4E1B1E01C935E
:1033F0000E94202DAEE1B1E01C930E94202DAFE190
:10340000B1E01C930E94202DA0E2B1E01C930E9429
:103410001E2DA1E2B1E01C930E94F82C80912001A6
:103420008093250196E0A5E2B1E00E940328009177
:1034300025010F938CE00E94C227482F0F91040FA3
:10344000A5E2B1E00C93E894A0E2B1E08C9187F999
:103450008C93E894A0E2B1E08C9186F98C938091F2
:1034600021018093230195E0A3E2B1E00E940328AB
:10347000E894A1E2B1E08C9187F98C93E894A1E201
:10348000B1E08C9186F98C93E894A1E2B1E08C9143
:1034900085F98C93AFE1B1E08C91AFE2B1E00E948D
:1034A000B727AFE2B1E00E941227EAE5FDE50E94EE
:1034B000A52B0E94F527AEE1B1E08C91AFE2B1E01F
:1034C0000E9412270E94B727AFE2B1E00E941227A4
:1034D000EAE5FDE50E94A52B0E94F527A4E1B1E0F5
:1034E0008C91AFE2B1E00E9412270E94B727A8E3B7
:1034F000B1E0ECE5FDE50E94A52B0E94F527A5E2D1
:10350000B1E08C91A8E3B1E00E9412270E94B72796
:10351000A8E3B1E00E941227E0E6FDE50E94A52B9A
:103520000E94F527A1E2B1E08C91A8E3B1E00E94EE
:1035300012270E94B727A8E3B1E00E941227E0E615
:10354000FDE50E94A52B0E94F527A0E2B1E08C9139
:10355000A8E3B1E00E9412270E94B727A4E1B1E0DE
:103560009C910E94C927A4E1B1E08C93AEE1B1E047
:103570009C910E94C927AEE1B1E08C93AFE1B1E02C
:103580009C910E94C927AFE1B1E08C93A5E2B1E024
:103590009C910E94C927A5E2B1E08C93A0E2B1E022
:1035A0009C910E94C927A2E2B1E08C93A3E2B1E012
:1035B0009C910E94C927A3E2B1E08C93A1E2B1E003
:1035C0009C910E94C927A4E2B1E08C93AFE1B1E0E5
:1035D0000D9111274CE350E00E94EB27AEE5B1E0DE
:1035E0000D931C93AEE5B1E00D911C91AEE1B1E0FD
:1035F0004D915527040F151FAEE5B1E00D931C93B7
:103600000895A4E1B1E08C910E94C227A6E2B1E046
:103610008C93AEE1B1E08C910E94C227A7E2B1E0A9
:103620008C93AFE1B1E08C910E94C227A8E2B1E097
:103630008C93A5E2B1E08C918C508C93A5E2B1E023
:103640008C910E94C227AEE2B1E08C9396E0AEE28C
:10365000B1E00E94FB27A2E2B1E08C910E94C22758
:10366000ABE2B1E08C9300912E0140912B01042B31
:10367000A9E2B1E00C93A3E2B1E08C910E94C227D1
:10368000ACE2B1E08C9395E0ACE2B1E00E94FB27A4
:10369000A4E2B1E08C910E94C227ADE2B1E08C932C
:1036A00000912C0140912D01042BAAE2B1E00C9372
:1036B0000E94E92C10EA0E94012D12E00E94012DC7
:1036C000A6E2B1E01C910E94012DA7E2B1E01C919D
:1036D0000E94012DA8E2B1E01C910E94012DA9E2F7
:1036E000B1E01C910E94012DAAE2B1E01C910E9460
:1036F000012D0E94F82C08950091DB0141E0041B8C
:10370000ACEDB1E00C93ACEDB1E00C9148E0049F5E
:103710000C92ACEDB1E08C918F5F8C93ACEDB1E08D
:10372000EC91FF27AAE4B1E091E07BE70E94452CF1
:1037300080914A01ACEDB1E0AD90BB24A2E8B1E0CC
:10374000AA0DBB1D8C93ACEDB1E08C918F5F8C9377
:10375000ACEDB1E0EC91FF27ABE4B1E091E07BE7A9
:103760000E94452C80914B01ACEDB1E0AD90BB24A3
:10377000A2E8B1E0AA0DBB1D8C93ACEDB1E08C9139
:103780008F5F8C93ACEDB1E0EC91FF27ACE4B1E03E
:1037900091E07BE70E94452C80914C01ACEDB1E0BB
:1037A000AD90BB24A2E8B1E0AA0DBB1D8C93ACED9B
:1037B000B1E08C918F5F8C93ACEDB1E0EC91FF2781
:1037C000ADE4B1E091E07BE70E94452C80914D0192
:1037D000ACEDB1E0AD90BB24A2E8B1E0AA0DBB1DF9
:1037E0008C93ACEDB1E08C918F5F8C93ACEDB1E03C
:1037F000EC91FF27AEE4B1E091E07BE70E94452C1D
:1038000080914E01ACEDB1E0AD90BB24A2E8B1E0F7
:10381000AA0DBB1D8C93ACEDB1E08C918F5F8C93A6
:10382000ACEDB1E0EC91FF27AFE4B1E091E07BE7D4
:103830000E94452C80914F01ACEDB1E0AD90BB24CE
:10384000A2E8B1E0AA0DBB1D8C93ACEDB1E08C9168
:103850008F5F8C93ACEDB1E0EC91FF27A0E5B1E078
:1038600091E07BE70E94452C80915001ACEDB1E0E6
:10387000AD90BB24A2E8B1E0AA0DBB1D8C93ACEDCA
:10388000B1E08C918F5F8C93ACEDB1E0EC91FF27B0
:10389000A1E5B1E091E07BE70E94452C80E0ACED32
:1038A000B1E0AD90BB24A2E8B1E0AA0DBB1D8C93A2
:1038B000089581E08093DE0180E08093E60188E056
:1038C00080937D014091060100917D01041718F05D
:1038D00011F00C94711DADE7B1E0AD90BB24A2E8EE
:1038E000B1E0AA0DBB1D0C91013011F00C947D1CB0
:1038F000A6EEB1E08C918F5F8C930091DE010130D8
:1039000011F00C94941CADE7B1E0AD90BB24A2E89B
:10391000B1E0AA0DBB1D8C9180FBA5E2B0E08C91BB
:1039200080F98C930C94641D023011F00C94A91C46
:10393000ADE7B1E0AD90BB24A2E8B1E0AA0DBB1D9C
:103940008C9180FBA5E2B0E08C9181F98C930C9472
:10395000641D033011F00C94BE1CADE7B1E0AD90D6
:10396000BB24A2E8B1E0AA0DBB1D8C9180FBA5E2AF
:10397000B0E08C9183F98C930C94641D043011F0A9
:103980000C94D31CADE7B1E0AD90BB24A2E8B1E04C
:10399000AA0DBB1D8C9180FBABE2B0E08C9180F94D
:1039A0008C930C94641D053011F00C94E81CADE769
:1039B000B1E0AD90BB24A2E8B1E0AA0DBB1D8C9193
:1039C00080FBABE2B0E08C9181F98C930C94641D88
:1039D000063011F00C94FD1CADE7B1E0AD90BB24B6
:1039E000A2E8B1E0AA0DBB1D8C9180FBABE2B0E078
:1039F0008C9182F98C930C94641D073011F00C9417
:103A0000121DADE7B1E0AD90BB24A2E8B1E0AA0D74
:103A1000BB1D8C9180FBABE2B0E08C9183F98C9361
:103A20000C94641D083011F00C94271DADE7B1E033
:103A3000AD90BB24A2E8B1E0AA0DBB1D8C9180FB28
:103A4000ABE2B0E08C9184F98C930C94641D093046
:103A500011F00C943C1DADE7B1E0AD90BB24A2E8A1
:103A6000B1E0AA0DBB1D8C9180FBABE2B0E08C9164
:103A700086F98C930C94641D0A3011F00C94511D3E
:103A8000ADE7B1E0AD90BB24A2E8B1E0AA0DBB1D4B
:103A90008C9180FBA8E2B0E08C9183F98C930C941C
:103AA000641D0B3011F00C94641DADE7B1E0AD90D6
:103AB000BB24A2E8B1E0AA0DBB1D8C9180FBA2E261
:103AC000B0E08C9181F98C93AEEDB1E08C918F5F79
:103AD0008C93ADE7B1E08C91885F8C9310F40C94DB
:103AE000621C0091E601003018F011F00C947A1D70
:103AF0000C94881D0091F401003011F00C94851D88
:103B0000119A8CE291E00E94DC27109A0C94941D8B
:103B100010980091F401003011F00C94941D8CE287
:103B200091E00E94DC2711980895A4E1B2E08C9105
:103B30008F5F8C930E94591CE3E0F1E0D190E0800C
:103B40008FEFE7FE8827F82E082F0E946D280E942D
:103B50009F28E6E7FAE50E94A52B0E94A9290E946A
:103B60004229EDE0F0E0ABEEB1E00E94362CEAE74E
:103B7000FAE50E94A52B0E94B229EBEEF1E00E942B
:103B800049280E941029EDE0F0E0ABEEB1E00E9480
:103B9000362CEBEEF1E00E940B28AFEEB1E0DC92A8
:103BA0000091F101013081E009F080E08F930091F4
:103BB000E7010F3080E010F009F081E09F91892348
:103BC000882311F40C94EB1D70917C017064709348
:103BD0007C010C94F01D70917C017F7B70937C01C3
:103BE0004091EF0100911402041718F011F00C94A9
:103BF000821F8FE711E00E943C27AFE2B1E00E94F4
:103C00001B27E4E4FCE50E94A52B0E942627A8E3DD
:103C1000B1E00E941B278FEB11E00E943C2709E0D6
:103C20000E9421278FEB1CE00E943C27009123017A
:103C3000003011F00C94361EECE9FDE50E94A52B36
:103C40000E94262786E00E949027E4ECFEE50E9471
:103C5000A52B0E94262785E00E949027E8ECFEE530
:103C60000E94A52B0E9426270C94A91E013011F05A
:103C70000C94421EEEECFEE50E94A52B0E94262726
:103C80000C94A91E023011F00C944E1EE8EDFEE5D6
:103C90000E94A52B0E9426270C94A91E033011F028
:103CA0000C94751EE2EEFEE50E94A52B0E942627CD
:103CB00087E00E949027E6EEFEE50E94A52B0E9479
:103CC000262785E00E949027E8EEFEE50E94A52BBE
:103CD0000E94262785E00E949027ECEEFEE50E94D8
:103CE000A52B0E9426270C94A91E043011F00C94D9
:103CF0008A1EE4EBFDE50E94A52B0E94262786E0A4
:103D00000E949027EEEEFEE50E94A52B0E9426273A
:103D10000C94A91E053011F00C94961EE6EFFEE5FA
:103D20000E94A52B0E9426270C94A91E063011F094
:103D30000C94A91EE0E0FFE50E94A52B0E94262717
:103D400084E00E949027E4E0FFE50E94A52B0E94FA
:103D500026278FEB1BE00E943C27E8EFFBE50E9443
:103D6000A52B0E94262783E91BE00E943C27E8EF51
:103D7000FBE50E94A52B0E94262781E08093DE01AF
:103D800088E080937D014091060100917D01041738
:103D900018F011F00C94321F83E9AEEDB1E01C91E4
:103DA0000E943C27ADE7B1E0AD90BB24A2E8B1E0B2
:103DB000AA0DBB1D0C91013011F00C940D1F009148
:103DC000DE010A3010F40C94031F0091DE014AE07A
:103DD0000E945D2CA6EFB1E08C93A8EAB0E4E6EF78
:103DE000F1E00E94CB2B0E9419278FEBAEEDB1E0E2
:103DF0001C910E943C27EAE0FFE50E94A52B0E944F
:103E000026270C940B1FA8EAB0E4EEEDF1E00E9427
:103E1000CB2B0E9419270C94251FECE0FFE50E9494
:103E2000A52B0E9426270091DE010A3010F40C9485
:103E3000251F8FEBAEEDB1E01C910E943C27E8EF0F
:103E4000FBE50E94A52B0E942627AEEDB1E08C91E8
:103E50008F5F8C93ADE7B1E08C91885F8C9310F409
:103E60000C94C31E0091F401003011F00C94411F1A
:103E700083E91CE00E943C2709E00E9421270C9462
:103E8000481F83E91DE00E943C2708E00E9421278B
:103E900083ED1FE00E943C270091F101013011F0F9
:103EA0000C94721FACE7B1E08C9186FB16F00C9479
:103EB000611FEEE0FFE50E94A52B0E9426270C94CF
:103EC000701FE6E1FFE50E94A52B0E94262784E0F3
:103ED0000E949027EAE1FFE50E94A52B0E94262779
:103EE0000C94751F06E00E9421270E94C4230091B4
:103EF0001402083711F00C94801F80E080931402A4
:103F00000C94F81F80911F01809307010E94F91FF4
:103F100081E08093130180910C01809312010E9433
:103F2000422085E08093130180911101809312015A
:103F30000E944220A3E1B1E08C918C5F8C930E949F
:103F40002B2380911E01809307010E94F91F8BE0B3
:103F50008093130180910C01809312010E944220F2
:103F60008FE08093130180911101809312010E94D0
:103F70004220A5E1B1E0E4E1F1E00E94CB2BE5E1D4
:103F8000F1E0A8EAB0E40E94312CE8EAF0E4A5E10F
:103F9000B1E01127222702E033270E94022A8FE78F
:103FA00013E10E943C27A5E1B1E00E941B278FEBA3
:103FB00013E10E943C2702E00E94212783E913E1DC
:103FC0000E943C2702E00E94212783ED13E10E941A
:103FD0003C2702E00E94212700911402083718F0C4
:103FE00011F00C94F51F0C94F81F80E080931402DC
:103FF0000895EEE7FAE50E94A52B0E94B229E7E0BA
:10400000F1E0D080EE24FF2400270E946D280E945A
:10401000BA28EDE0F0E0A8E0B1E00E94362CE8E03C
:10402000F1E00E949C2CEDE0F0E00E940B28ACE057
:10403000B1E0DC92E8E0F1E00E947D2CEDE0F0E000
:10404000ADE0B1E00E94362CEEE7FAE50E94A52B28
:104050000E94B229EDE0F1E00E9449280E94102957
:10406000EDE0F0E0ADE0B1E00E94362CEDE0F1E0F3
:104070000E94DB2CEDE0F0E00E940B28A1E1B1E012
:10408000DC92089500911201003011F00C94902000
:104090008FE7A3E1B1E01C910E943C2782E00E94DF
:1040A000902780E00E94902782E00E94902701E004
:1040B0000E9421278FEBA3E1B1E01C910E943C27D5
:1040C00082E00E94902701E00E94212782E00E9466
:1040D000902701E00E94212783E9A3E1B1E01C9130
:1040E0000E943C2782E00E94902701E00E94212745
:1040F00082E00E94902701E00E94212783EDA3E146
:10410000B1E01C910E943C2782E00E94902781E050
:104110000E94902782E00E94902701E00E942127C0
:1041200000911201013011F00C94C6208FE7A3E139
:10413000B1E01C910E943C2782E00E94902703E09E
:104140000E9421278FEBA3E1B1E01C910E943C2744
:1041500082E00E94902703E00E94212783E9A3E1E7
:10416000B1E01C910E943C2782E00E94902703E06E
:104170000E94212783EDA3E1B1E01C910E943C271E
:1041800082E00E94902703E00E9421270091120103
:10419000023011F00C9414218FE7A3E1B1E01C91DF
:1041A0000E943C2780E00E94902780E00E94902798
:1041B00082E00E94902701E00E9421278FEBA3E17B
:1041C000B1E01C910E943C2781E00E94902781E091
:1041D0000E94902782E00E94902701E00E94212700
:1041E00083E9A3E1B1E01C910E943C2782E00E9498
:1041F000902780E00E94902780E00E94902701E0B5
:104200000E94212783EDA3E1B1E01C910E943C278D
:1042100082E00E94902781E00E94902781E00E9426
:10422000902701E00E94212700911201033011F034
:104230000C9462218FE7A3E1B1E01C910E943C271E
:1042400080E00E94902780E00E94902782E00E94F8
:10425000902701E00E9421278FEBA3E1B1E01C91A0
:104260000E943C2781E00E94902781E00E949027D5
:1042700082E00E94902701E00E94212783E9A3E1C8
:10428000B1E01C910E943C2780E00E94902780E0D2
:104290000E94902782E00E94902701E00E9421273F
:1042A00083EDA3E1B1E01C910E943C2781E00E94D4
:1042B000902781E00E94902782E00E94902701E0F1
:1042C0000E94212700911201043011F00C94AD21BD
:1042D0008FE7A3E1B1E01C910E943C2782E00E949D
:1042E000902701E00E94212782E00E94902701E0B0
:1042F0000E9421278FEBA3E1B1E01C910E943C2793
:1043000082E00E94902781E00E94902782E00E9434
:10431000902701E00E94212783E9A3E1B1E01C91ED
:104320000E943C2780E00E94902780E00E94902716
:1043300082E00E94902701E00E94212783EDA3E103
:10434000B1E01C910E943C2702E00E94212782E0FC
:104350000E94902701E00E94212700911201053060
:1043600011F00C94FB218FE7A3E1B1E01C910E94B6
:104370003C2782E00E94902780E00E94902780E006
:104380000E94902701E00E9421278FEBA3E1B1E07A
:104390001C910E943C2782E00E94902781E00E94AD
:1043A000902781E00E94902701E00E94212783E965
:1043B000A3E1B1E01C910E943C2780E00E9490277D
:1043C00080E00E94902782E00E94902701E00E94F6
:1043D000212783EDA3E1B1E01C910E943C2781E0FD
:1043E0000E94902781E00E94902782E00E949027FF
:1043F00001E00E94212700911201063011F00C9477
:1044000049228FE7A3E1B1E01C910E943C2782E0A2
:104410000E94902780E00E94902780E00E949027D1
:1044200001E00E9421278FEBA3E1B1E01C910E94E3
:104430003C2782E00E94902781E00E94902781E043
:104440000E94902701E00E94212783E9A3E1B1E0C7
:104450001C910E943C2782E00E94902780E00E94ED
:10446000902782E00E94902701E00E94212783ED9F
:10447000A3E1B1E01C910E943C2782E00E949027BA
:1044800081E00E94902782E00E94902701E00E9434
:10449000212700911201073011F00C948E228FE732
:1044A000A3E1B1E01C910E943C2780E00E9490278C
:1044B00080E00E94902782E00E94902701E00E9405
:1044C00021278FEBA3E1B1E01C910E943C2702E081
:1044D0000E94212782E00E94902701E00E9421276C
:1044E00083E9A3E1B1E01C910E943C2702E00E9415
:1044F000212782E00E94902701E00E94212783ED7E
:10450000A3E1B1E01C910E943C2702E00E94212718
:1045100082E00E94902701E00E9421270091120171
:10452000083011F00C94DC228FE7A3E1B1E01C917C
:104530000E943C2782E00E94902780E00E94902702
:1045400082E00E94902701E00E9421278FEBA3E1E7
:10455000B1E01C910E943C2782E00E94902781E0FC
:104560000E94902782E00E94902701E00E9421276C
:1045700083E9A3E1B1E01C910E943C2782E00E9404
:10458000902780E00E94902782E00E94902701E01F
:104590000E94212783EDA3E1B1E01C910E943C27FA
:1045A00082E00E94902781E00E94902782E00E9492
:1045B000902701E00E94212700911201093011F09B
:1045C0000C942A238FE7A3E1B1E01C910E943C27C1
:1045D00082E00E94902780E00E94902782E00E9463
:1045E000902701E00E9421278FEBA3E1B1E01C910D
:1045F0000E943C2782E00E94902781E00E94902741
:1046000082E00E94902701E00E94212783E9A3E134
:10461000B1E01C910E943C2780E00E94902780E03E
:104620000E94902782E00E94902701E00E942127AB
:1046300083EDA3E1B1E01C910E943C2781E00E9440
:10464000902781E00E94902782E00E94902701E05D
:104650000E94212708958FE7A3E1B1E01C910E94F9
:104660003C2702E00E9421278FEBA3E1B1E01C91DF
:104670000E943C2780E00E94902701E00E942127B1
:1046800083E9A3E1B1E01C910E943C2781E00E94F4
:10469000902701E00E94212783EDA3E1B1E01C9166
:1046A0000E943C2702E00E942127089587E0E9E26A
:1046B0000E944F2A5CEC87E0E9E20E94772A54E4EA
:1046C00087E0E9E20E94772A089587E0E9E20E9404
:1046D0004F2A87E0E9E2A4E0B2E00E947C2B5EEB87
:1046E00087E0E9E20E94772A87E0A9EFB1E0E9E2FA
:1046F00022E02A930E949F2A87E0E9E20E944F2A43
:1047000087E0E9E2ACE0B2E00E947C2B5EEB87E060
:10471000E9E20E94772A87E0A2E0B2E0E9E222E043
:104720002A930E949F2AA9EFB1E00D911C914AE0C3
:1047300050E00E94EB27A9EFB1E00D931C93A9EF85
:10474000B1E00D911C9140E150E00E94D826A9EF04
:10475000B1E04D935C93A2E0B2E00D911C914AE070
:1047600050E00E94EB27A2E0B2E00D931C93A2E080
:10477000B2E00D911C9140E150E00E94D826A2E0E9
:10478000B2E04D935C930895ACE7B1E08C9185FB6A
:1047900016F00C94DA2383ED11E00E943C27EEE141
:1047A000FFE50E94A52B0E94262709E00E942127F1
:1047B0000C946524AEE7B1E04D915C91A9EFB1E0B6
:1047C0000D911C91041715070CF402C00C940B24D6
:1047D000A9EFB1E00D911C91003050E0150781E088
:1047E00009F480E08F93A9EFB1E00D911C9102359F
:1047F00053E0150781E009F480E09F918923882325
:1048000011F40C940B24A9EFB1E08D919C91AEE7CB
:10481000B1E08D939C93A0E8B1E04D915C91A9EF3C
:10482000B1E00D911C91041715071CF011F00C94C8
:104830001B240C943E24A9EFB1E00D911C91003093
:1048400050E0150781E009F480E08F93A9EFB1E013
:104850000D911C91023553E0150781E009F480E0C9
:104860009F918923882311F40C943E24A9EFB1E091
:104870008D919C91A0E8B1E08D939C93ABEFB1E05A
:10488000E9EFF1E00E94C42BEBEFF1E0A8EAB0E41D
:104890000E94312CE8EAF0E4ABEFB1E011272227C7
:1048A00003E031E00E94022A83ED11E00E943C27E0
:1048B000ABEFB1E00E941B2783E00E949027E6E265
:1048C000FFE50E94A52B0E942627ACE7B1E08C9162
:1048D00084FB16F00C947B2483ED18E00E943C27A7
:1048E000EAE2FFE50E94A52B0E94262709E00E942C
:1048F00021270C940625AEE7B1E04D915C91A9EF1C
:10490000B1E00D911C91041715070CF402C00C9432
:10491000AC24A9EFB1E00D911C91003050E01507D7
:1049200081E009F480E08F93A9EFB1E00D911C9133
:10493000023553E0150781E009F480E09F91892357
:10494000882311F40C94AC24A9EFB1E08D919C91D3
:10495000AEE7B1E08D939C93A0E8B1E04D915C91FE
:10496000A9EFB1E00D911C91041715071CF011F08F
:104970000C94BC240C94DF24A9EFB1E00D911C91A0
:10498000003050E0150781E009F480E08F93A9EF33
:10499000B1E00D911C91023553E0150781E009F457
:1049A00080E09F918923882311F40C94DF24A9EFE0
:1049B000B1E08D919C91A0E8B1E08D939C93ABEF19
:1049C000B1E0E2E0F2E00E94C42BEBEFF1E0A8EAF4
:1049D000B0E40E94312CE8EAF0E4ABEFB1E011273B
:1049E000222703E031E00E94022A83ED18E00E94B2
:1049F0003C27ABEFB1E00E941B2783E00E94902789
:104A0000E2E3FFE50E94A52B0E94262708950F925E
:104A10001F922F923F924F925F927F92AF92BF92DE
:104A20000F931F932F933F934F935F936F937F93B6
:104A30008F939F93AF93BF93CF93DF93EF93FF93A6
:104A40008FB78F938BB78F9388278BBFA2E8B1E086
:104A50008C918F5F8C93329B0C94312580E08093F6
:104A6000E70180E080935901009182010E3111F03D
:104A70000C948E260091E701043110F00C9445252A
:104A8000A7EEB1E08C918F5F8C9370916E007E7F6A
:104A900070936E000091DD0141E0041BACEDB1E0CC
:104AA0000C93ACEDB1E00C9148E0049F0C92ACED9E
:104AB000B1E0AD90BB24A3E8B1E0AA0DBB1D8C9181
:104AC00080935201ACEDB1E0AD90BB24A4E8B1E01D
:104AD000AA0DBB1D8C9180935301ACEDB1E0AD905C
:104AE000BB24A5E8B1E0AA0DBB1D8C9180935401B5
:104AF000ACEDB1E0AD90BB24A6E8B1E0AA0DBB1DC2
:104B00008C9180935501ACEDB1E0AD90BB24A7E84A
:104B1000B1E0AA0DBB1D8C9180935601ACEDB1E0C4
:104B2000AD90BB24A8E8B1E0AA0DBB1D8C91809389
:104B30005701ACEDB1E0AD90BB24A9E8B1E0AA0DFE
:104B4000BB1D8C9180935801A3E5B1E00D91112715
:104B50004CE350E00E94EB27AAE5B1E00D931C93D3
:104B6000AAE5B1E00D911C91A4E5B1E04D91552766
:104B7000040F151FAAE5B1E00D931C93A5E5B1E064
:104B80000D9111274CE350E00E94EB27ACE5B1E01A
:104B90000D931C93ACE5B1E00D911C91A6E5B1E03D
:104BA0004D915527040F151FACE5B1E00D931C93F3
:104BB00000915201013011F00C94452600915801EA
:104BC000003011F00C940F26AAE5B1E04D915C91F4
:104BD000AEE5B1E00D911C910417150780E00CF0D3
:104BE00081E08F93ACE5B1E04D915C91AEE5B1E031
:104BF0000D911C910417150780E00CF481E09F9142
:104C00008923882311F40C940A2681E080935901AA
:104C10000C940D2680E0809359010C944326AAE55C
:104C2000B1E04D915C91AEE5B1E00D911C9104179E
:104C3000150780E00CF081E08F93ACE5B1E04D9179
:104C40005C91AEE5B1E00D911C910417150780E071
:104C50000CF481E09F9189238F934091230100916F
:104C60005701041781E009F080E09F918923882390
:104C700011F40C94402681E0809359010C94432652
:104C800080E0809359010C94482680E0809359017C
:104C9000ACE7B1E08C9186FB81E00EF080E08F9371
:104CA0000091F101013081E009F080E09F918923BA
:104CB000882311F40C94682680E0ACEDB1E0AD904F
:104CC000BB24AAE8B1E0AA0DBB1D8C930C947326FB
:104CD00080915901ACEDB1E0AD90BB24AAE8B1E000
:104CE000AA0DBB1D8C93ADEDB1E08C918F5F8C93C1
:104CF000409105010091DD01041718F011F00C94AA
:104D000083260C94862681E08093DD0181E08093E8
:104D1000820170916E00716070936E008F918BBFF5
:104D20008F918FBFFF91EF91DF91CF91BF91AF91A5
:104D30009F918F917F916F915F914F913F912F91B3
:104D40001F910F91BF90AF907F905F904F903F90D9
:104D50002F901F900F901895F894FFCF31003200DC
:104D60003300340035003600370038003900313068
:104D7000002A00535A004D535A000102030405064D
:104D80000708090A0D0F1200ED91FC91EF5FFF4F2C
:104D9000FC93EE930895ED91FC91E150F040FC936B
:104DA000EE93089509D00E94EB2700FC10D00895DF
:104DB00003D01ED001F8F9CF0024E89457FF02C0B9
:104DC00009D0689400F80BD010F80124089502D09F
:104DD00009D00895509540954F5F5F4F0895E8942E
:104DE00017FF0895009510950F5F1F4F6894089561
:104DF000352F242FE894452B11F468940895512FF2
:104E0000402F0027112780E1440F551F001F111F5D
:104E1000021B130B416018F4020F131F4E7F8A957B
:104E200099F708958F938D918823E9F711978F91C2
:104E30000895A8EAB0E48D91882311F071D0FBCFDA
:104E4000089580E26DD00A95E1F708950E949F29A8
:104E5000802D11F065D0FACF089581E067D015D08C
:104E600080E864C08FE7213039F08FEB223021F0E9
:104E700083E9233009F083ED810F0C94962788EEA7
:104E800093E09AD03197D9F7089583E0992794C099
:104E90008AEF90E00E94DC270F9A0E9A0D9A0C9AE6
:104EA0000B9A0A9A129885E090E00E94DC271398EA
:104EB00017981698159A149A139AEF93FF93ECE8A3
:104EC000F1E00E94D027FF91EF91139872D0139ACE
:104ED000EF93FF93ECE8F1E00E94D027FF91EF9170
:104EE000139867D0139AEF93FF93ECE8F1E00E94D8
:104EF000D027FF91EF9113985CD01498139AEF93F9
:104F0000FF93ECE8F1E00E94D027FF91EF91139816
:104F100050D088E20BD08EE009D086E007D008950B
:104F2000129A829505D004D044D008951298F9CFF2
:104F3000859510F4149A01C01498859510F4159A6B
:104F400001C01598859510F4169A01C0169885959C
:104F500010F4179A01C01798139AEF93FF93ECE897
:104F6000F1E00E94D027FF91EF9113980895982FB8
:104F700082958F70805D8D939F70905D9D93882743
:104F80008C9308954AE0082F0E945D2C0295802B97
:104F90000895892F8F70905110F0865FFCCF08958F
:104FA0003197F1F70895689462F80895E89462F8EB
:104FB000089581E090E000C0EF93FF93EE27E82B87
:104FC000E92B31F0E0EAFFE03197F1F70197D1F7F3
:104FD000FF91EF9108950F92B801469F8001479F7E
:104FE000100D569F100D0F9008950E949F290D924D
:104FF0000020D9F70895903029F08C91880F9A9568
:10500000E9F78C930895903029F08C9186959A95C4
:10501000E9F78C9308953DD0992711278F2D880F9C
:1050200080E8F82A802F881F08F41FEF41F08F577F
:10503000082F07FD04C0003240F08FEF01C0882721
:10504000982FD82EE82EF82E09C08FE1801B082F4C
:10505000F694E794D79497950A95D1F7112351F0D8
:105060009095D094E094F09481E0980F8827D81E12
:10507000E81EF81E0F2DFE2CED2CD92E0895D0948D
:10508000E094F09491E0D90E9927E91EF91E10954D
:105090000895D190E190F19001910895219131917D
:1050A000419151910895102F90E8FF0C001F09279E
:1050B000990FF7941078652F90E8440F551F5927E2
:1050C000990F4795607800380895FF0C90E8902775
:1050D000110F9795F794092F0895102FBD2CDE2CF2
:1050E000EF2CF02E11234AF4B094D094E094F09475
:1050F0009FEFB91AD90AE90AF90A0EE1FF2039F43B
:10510000FE2CED2CDB2CBB240850C2F767C032F01C
:105110000A95BB0CDD1CEE1CFF1CF9CF0E949128E8
:10512000D4CFB7FE089590E8B91611F4D0FE0895D3
:105130009FEFD91AE90AF90A09F403950895502F47
:105140002D2D3E2D4F2D612F08952DEC3CEC4CEC78
:105150005DE366270FC09DDFF2DFDD24EE2490E8DB
:10516000F92E0FE307C09ADF05C02227332740E25C
:1051700051E46627552351F1002381F194DF71F149
:105180001627005850580894050B18F407FD03C063
:1051900025C007FD23C0469537952795F694E794DB
:1051A000D79422D0FF202AF0DD0CEE1CFF1C01500A
:1051B00073F09D2D969548F0DD203AF4EE202AF408
:1051C00091E0D90E9927E91EF91E7FCF07C09FE70E
:1051D000092FF92A9FEFD92EE92E0895DD24EE2418
:1051E000FF240027112708959F929924AA24BB2405
:1051F00088E1D216E306F40628F0D21AE30AF40A8C
:10520000089401C08894991CAA1CBB1CDD0CEE1CE0
:10521000FF1C8A9571F7D92CEA2CFB2C9F900895DE
:1052200042DFE1F25038D1F2162700585058089466
:10523000051F12F418F4CBCF08F0D0CF0BD0FF200D
:105240002AF0BB0CDD1CEE1CFF1C3FCF0F5F0BF4E4
:10525000BECF3BCF9F929924AA24BB24992788E1F3
:10526000990CAA1CBB1CDD1CEE1CFF1C30F4920E1A
:10527000A31EB41ED91EE91EF91E8A9589F79F90B8
:1052800008950CDF10DF503829F090E869270CC032
:105290000AF045D01ACF5FE322273327442701C005
:1052A000FDDE01DF5038B1F3003899F3902F951BE4
:1052B0008BF312F434D0FACF983118F02227332729
:1052C0004427983028F0232F342F44279850F9CFC3
:1052D000992329F04695379527959A95D9F7912FD7
:1052E000962742F014D0B0F6F794E794D7940F5F66
:1052F0008BF66DCF10D051F008F4C1DEFF2052F2D2
:10530000DD0CEE1CFF1C0150CBF761CF67CFD20E36
:10531000E31EF41E0895D21AE30AF40A0895DF92F8
:10532000EF92FF920F931F93D22EE32EF42E052FB0
:10533000162F6F915F914F913F912F910895D895BE
:10534000319628F48F938BB783958BBF8F91002074
:105350000895F5DFD02CF3DFE02CF1DFF02CEFDF48
:10536000002D0895ECDF202DEADF302DE8DF402D01
:10537000E6DF502D089507FB00680EF40F7757FB0A
:1053800050680EF45F7707FD02C057FF05C0D216C4
:10539000E306F406050708952D153E054F05500751
:1053A000089591E005C092E003C094E001C098E048
:1053B000C6DF0D929A95E1F70895E80FF91F01D025
:1053C000F0CF28F48F938BB783958BBF8F9108957F
:1053D000882311F4992329F00E949F29E9F7019766
:1053E000D9F7089591E0882321F08894991F8A9530
:1053F000E9F7892F90950895883018F01196885014
:10540000FBCF08952E2E3F2E992781918D3209F0E2
:1054100093958823D1F79A95E22DF32D112361F00E
:10542000091718F011F0101B01C0191B28F021F00A
:1054300080E28D931A95E9F780818D3219F48D936E
:10544000319604C0222311F08BE28D93091738F0B6
:1054500031F0091B21F080E38D930A95E9F78191E2
:105460008D938823E1F7332351F0EA2FFB2F3196F8
:1054700033958E9182933A95E1F78EE28C9308955D
:105480000181082B0183128119231283EF93FF936B
:10549000E4E1F0E00E94D027FF91EF9108950E948F
:1054A000D627FF270E94F229EBDFEF93FF93ECE76B
:1054B000F7E00E94D027FF91EF91182B1283092368
:1054C0000183EF93FF93E4E1F1E00E94D027FF9185
:1054D000EF911081182311F00E94D327EF93FF93CF
:1054E000E4E6F6E00E94D027FF91EF9108950E9434
:1054F000F229FF2721E048E006C00E94F229FF2799
:1055000029915D9148E0BCDF579510F4182B128368
:10551000EF93FF93E4EDF0E00E94D027FF91EF912D
:10552000182B1283EF93FF93E4E2F0E00E94D02760
:10553000FF91EF914A9539F72A9519F708950E943E
:10554000F229FF27299148E055279ADF0923018393
:10555000EF93FF93E0E2F0E00E94D027FF91EF91FC
:1055600088941081182309F008945795EF93FF93BE
:10557000E8EDF0E00E94D027FF91EF914A9529F7DE
:105580005D932A9501F708957BDF09230183EF934B
:10559000FF93E0E2F0E00E94D027FF91EF91E894C2
:1055A0001081182309F06894EF93FF93E8EDF0E081
:1055B0000E94D027FF91EF91089562DF16F4182B17
:1055C0001283EF93FF93E4EDF0E00E94D027FF9168
:1055D000EF91182B1283EF93FF93E4E2F0E00E9427
:1055E000D027FF91EF91089533273093190230931C
:1055F000160255DF0EF458C03091160230FD54C02B
:1056000066276093180263956093170221E050EFBC
:1056100048E079DFB9DF31F9B7DF32F9632F66701F
:10562000663009F441C0603019F031FB40D025C02C
:1056300060911702709119026717B1F0C0F48F934F
:105640009F93862F8A95AAE1B2E0D6DECBDE7C91CD
:1056500078236894772329F4E89460911702609383
:1056600018029F918F9109C0689421D006C0E894D8
:105670001ED060911702609318029FDF609117029D
:10568000639560931702613409F0C4CF60911802EA
:10569000609319026623E89409F4689430F9309312
:1056A0001602E89462F80895689462F808958F935A
:1056B0009F93AAE1B2E0809117028A959DDE92DE67
:1056C0007C9116F4782B01C079237C939F918F9164
:1056D00008958F9389DF8F91A0E0B0E056F0119686
:1056E0008F93AF93BF9385DFBF91AF918F910EF0F2
:1056F000F6CF0A2F1B2F0895AF93BF93EF93FF931D
:1057000038E0EAE1F2E00D9101933A95E1F7FF917B
:10571000EF9130E43093190233273093160269DF9A
:1057200038E0BF91AF91EAE1F2E00D9141910417A9
:1057300019F43A95D1F708950E94D32708950F934D
:1057400001E00BBF0F91889408950F930027F9CFC4
:105750000F9302E0F6CF0F9303E0F3CF000F111F7A
:10576000221F331F089500951095209530950F5FE7
:105770001F4F2F4F3F4F0895019110810EC001918F
:105780001191219130810BC00191108117FF05C04B
:105790003FEF2FEF04C0008111272227332737FF67
:1057A00003C0E1DF8DE28D93CF93DF93CF92DF9241
:1057B000EF92AA24BB24CC24DD24EE2440E2CAE0EC
:1057C000DD2755E093E38881890F87FD9F7083FD76
:1057D000907F891B89935A95A9F7C0DFAA1CBB1C2F
:1057E000CC1CDD1CEE1C4A9551F7E894EFE0FF2736
:1057F00082910ED0EB30E0F71EF068948A2D0CD029
:1058000088278D93EF90DF90CF90DF91CF9108950F
:10581000982F829501D0892F8F70805D26F080337C
:1058200009F4089568948D93089541E003C042E01F
:1058300001C044E0E40F8827F81F8291982F8295D9
:1058400006D0892F04D04A95C1F70C942E2C8F7066
:105850008A3008F0895F805D8D93089588278D9345
:10586000089581918D938823E1F7089594E08191C3
:105870008D939A95E1F70895F999FECFE1BDF2BDB8
:105880003196089591E001C092E07B3751F47FB7E3
:10589000F894F2DF8D9180BDFA9AF99A9A95C9F73A
:1058A0007FBF7727089591E001C092E0E5DFF89A85
:1058B00080B58D939A95D1F70895FF93881BF9E0F1
:1058C000001FFA9511F4FF910895881F841B18F4A6
:1058D000840F8894F5CF0894F3CF00276CE871917A
:1058E00098E00695779577FF18F477FD08F006277E
:1058F0009A95B9F78A9599F70895CBDBD4DB039590
:10590000AAF087E1DD0CEE1CFF1C8A9589F00A9550
:10591000CAF7FF205AF000240D280E280F28002077
:1059200039F00A95DD0CEE1CFF1CDAF70A95CDCB99
:1059300055CCAFDB80E003C0ACDB802F80788823C0
:1059400021F0DF92EF92FF920F938F93ACDB802FC9
:10595000839512F443DC1BC080958A95885E0AF417
:1059600015C088501AF40CD0D92210C0DD248850FC
:105970001AF406D0E9220AC0EE2402D0F92206C0A9
:105980009FEF8770990F8A95EAF708959EDB8F91B4
:105990008823D9F35F914F913F912F910F93EBDCC7
:1059A0000F9199F390F302D050687BCC5FE340E80D
:1059B0003327222708956DDB0F930F776CDCBDDF53
:1059C0008F918078082B089541984098399838989D
:1059D0000895389A399803D0389801D0399AEF93BE
:1059E000FF93E0E1F0E00E94D027FF91EF9108954E
:1059F000389A399AF4DF3898309BFECFF0DF399827
:105A0000EECF0894111F01C0110F69F0389A18F4F5
:105A10000000399802C0399A00C0E1DF3898309B05
:105A2000FECFDDDFF1CF389A3998D9DF3898309B37
:105A3000FECFE8943199689462F8D1CF089401C000
:105A40008894331F11E0389A3998C9DF3898309B11
:105A5000FECFC5DF889431990894111FA0F7389ABA
:105A6000379510F4399801C0399AB9DF3898309BCE
:105A7000FECFB5DF08950000C8429A99993F000013
:105A800020415A6F6E6120616461746F6B006265C2
:105A900074006C740000736500003D0045727A006C
:105AA0006B656C006B20737A00006D613A2000001A
:105AB0004E4F2053454E534F52203120202020205E
:105AC000000053454E534F52203120435243204F44
:105AD0004B20202020004944312000004552524FE5
:105AE00052204441544120312D5749524520200035
:105AF0004E4F2053454E534F52203220202020201D
:105B0000000053454E534F52203220435243204F02
:105B10004B20202020004944322000004552524FA3
:105B20005221205332202D20544F56414242000032
:105B30004B00737A6974657474653A0031342D30A2
:105B4000332D323031342032323A33363A3130006C
:105B500053545249435A2052414A4D554E442053C2
:105B60002E522E200000435A0000482056494B5424
:105B70004F5220432E562E2000004D454E55203EBC
:105B800020525443206265006C6C69742E20000022
:105B90004D454E55203E205A6F6E61207465737AD4
:105BA000742020004D454E55203E205A6F6E6120D6
:105BB000626500006C6C69742E004D454E55203EA8
:105BC000204265006C6C69740000736F6B202000CC
:105BD0004F5054203E204C4344206B6F6E747261D2
:105BE000737A74004F5054203E204E616779737A67
:105BF00000006D206964000020004F5054203E20BA
:105C000045730000727A00004F5054203E204D61D1
:105C10007374657220737A656C6570004F50542000
:105C20003E2042007669740020706F72742020203C
:105C300000004D454E55203E204F524120424541E7
:105C40004C4C0000202000003D3D00004D454E55CD
:105C5000203E2050455243204245414C4C200000FC
:105C60004D454E55203E204D50204245414C4C0064
:105C70004D454E55203E204556204245414C4C2036
:105C8000202020003D3D3D3D00004D454E55203E2D
:105C900020484F4E4150204245414C4C00004D455C
:105CA0004E55203E204E4150204245414C4C202034
:105CB00000004D454E55203E20484554204E415051
:105CC0004A414900484554464F003D3D3D3D3D0059
:105CD0004B4544440000535A4552444100003D3D69
:105CE0003D3D3D3D0000435355544F52544F4B00F2
:105CF0003D3D3D3D3D3D3D3D3D0050454E54454BB8
:105D00000000535A4F4D424154003D3D3D3D3D3D05
:105D10003D0056415341524E415000003D3D3D3DF6
:105D20003D3D3D3D00004D454E5453453F004947E4
:105D3000454E20204E454D003D3D3D002020454C28
:105D40004D454E545645202000004E494E435320A9
:105D5000454C4D454E54564520003A003230000027
:105D60002E005A4F4E412056414C41535A544153F4
:105D70003A005A6F6E613A200000496E616B746997
:105D80007600416B74697620202000004E617069B6
:105D900020202020200048657469280048007429CC
:105DA00000004B6564290000537A652900004373A5
:105DB0007529000050006E290000537A6F290000F9
:105DC00056617329000042653A004B693A00205A37
:105DD0004F4E4120414B5449563F00002E205A4F10
:105DE0004E41204759414B4F5249534147413F0093
:105DF0004E41504920204845544900002E205A6FFA
:105E00006E612062656B617063732E004E61706914
:105E100000004865746900002E205A6F6E61206B87
:105E2000696B617063732E002E206D656C79696BF0
:105E3000206E61706F6E3F004D454E5453454D3F8F
:105E400000004F5054203E204B6F6E747261737A85
:105E500074202020202000004B6F6E7472617374D8
:105E6000203D2000252020006D2020202020000043
:105E700020302500353025003130302500004E61BE
:105E80006779737A00006D203D2000002A00456E7E
:105E9000676564006C79657A76653F00537A656C56
:105EA000657020205A6F6E61000020706F72740060
:105EB0004E696E637320202B5A6F6E6120204574EB
:105EC000682E0000746600002020202000004B6532
:105ED0006464202020202000537A657264612020B1
:105EE0002000437300007400727400006B006E7435
:105EF000656B20202000537A6F6D62617420200052
:105F000056617300726E6170200031002D004E6585
:105F1000647665730000537A000072617A00543130
:105F20002E45727200004320000054322E457272DA
:045F3000000043002A
:00000001FF
